S01700006F70656E626C745F786D63343730302E73726563A7
S3150C0000004088FE1F010200089902000899020008A8
S3150C00001099020008990200089902000800000000E5
S3150C000020000000000000000000000000990200081B
S3150C00003099020008000000009902000899020008C5
S3150C0000409902000899020008990200089902000812
S3150C0000509902000899020008990200089902000802
S3150C00006099020008000000000000000000000000DB
S3150C0000709902000800000000990200089902000885
S3150C00008099020008990200089902000899020008D2
S3150C00009099020008990200089902000899020008C2
S3150C0000A099020008990200089902000899020008B2
S3150C0000B099020008990200089902000899020008A2
S3150C0000C09902000899020008990200089902000892
S3150C0000D09902000899020008990200089902000882
S3150C0000E09902000899020008990200089902000872
S3150C0000F09902000899020008990200089902000862
S3150C0001009902000899020008990200089902000851
S3150C0001109902000899020008990200089902000841
S3150C0001209902000899020008990200089902000831
S3150C0001309902000899020008990200089902000821
S3150C0001409902000899020008990200089902000811
S3150C0001509902000899020008990200089902000801
S3150C000160000000000000000000000000000000007D
S3150C00017099020008990200089902000899020008E1
S3150C00018099020008990200089902000899020008D1
S3150C00019099020008990200089902000899020008C1
S3150C0001A099020008990200089902000899020008B1
S3150C0001B099020008990200089902000899020008A1
S3150C0001C09902000899020008990200089902000891
S3150C0001D09902000899020008990200080000000024
S3150C0001E09902000899020008990200089902000871
S3150C0001F099020008000000009902000800000000A7
S3150C000200DFF874D01D4880471D4C1E4DAC4209DAF0
S3150C00021021686268A368043BA2BFC858D050FAE7AD
S3150C0002200C34F3E7184B194CA34208DA19685A68D0
S3150C0002300020043AA4BF8850FBE70833F4E71448BF
S3150C00024080471448804700008841000C4088FE1FF8
S3150C000250340000008841000C4088FE1F000000009E
S3150C0002607888FE1F1C110000000000200000000012
S3150C00027000000020A03000004088FE1F2905000861
S3150C00028048020008600200086002000878020008B4
S3150C000290E13F0008C13E0008FEE7000082B00023E3
S3150C0002A0019303E000BF019B01330193019B834241
S3150C0002B0F8D302B0704700BF72B60D4B0D4A9A6068
S3150C0002C0BFF34F8F62B6D3F8882042F47002C3F89E
S3150C0002D088205A6922F008025A61074941F2140231
S3150C0002E08B5823F00F0343F004038B50704700BF69
S3150C0002F000ED00E0000000080010005800487047B0
S3150C000300001BB70010B51E4BDB6813F4803F27D0DB
S3150C0003101C4BDB6813F0010F02D1FFF7EFFF00E077
S3150C0003201948184B1B6813F0040F11D015498A682D
S3150C000330C2F303628B68C3F306238C68C4F30644CA
S3150C000340611C02FB0112B0FBF2F203FB022208E075
S3150C0003500C4B9B6803F07F030133B0FBF3F200E018
S3150C000360094A0749C868C0B20130B2FBF0F3086904
S3150C00037000F001000130B3FBF0F0044B186010BD27
S3150C000380004600501047005000366E01C0FF032097
S3150C00039070B5574B1B6813F0010F09D1544A5368BB
S3150C0003A043F001035360524B1B6813F0010FFAD054
S3150C0003B0504B1B6813F4007F08D04E4A936843F4E5
S3150C0003C00073936041F64C50FFF768FF4A4C636824
S3150C0003D043F40023636040F6C410FFF75FFF6368C5
S3150C0003E023F4803323F002036360444B5B6813F001
S3150C0003F0300F21D0103C636823F4702323F03003B4
S3150C0004006360FFF77BFF3E4BA3FB00231B0D013BF9
S3150C000410626842EA03436360374BDA6822F00102F2
S3150C000420DA605A6822F400325A60334B1B6803F4C4
S3150C0004306073B3F5607FF8D12F4B5A6842F0010216
S3150C0004405A605A6842F010025A602E4A9A605A68EC
S3150C00045042F040025A605A6822F010025A605A68FA
S3150C00046042F480225A60244B1B6813F0040FFAD016
S3150C000470214A536823F0010353601F4B1B6813F08A
S3150C000480010FFAD1204C4FF00113E3600026666190
S3150C0004902661266266620323E3611C4BA3611C4B37
S3150C0004A0A362154D6B6823F040036B60194BAB6070
S3150C0004B04FF41660FFF7F2FE174BAB604FF461601A
S3150C0004C0FFF7ECFE154BAB604FF49650FFF7E6FECC
S3150C0004D0134BAB6041F27070FFF7E0FE114BAB6053
S3150C0004E04FF4E150FFF7DAFE6660FFF70BFF70BDC5
S3150C0004F00042005000440050104700500047005086
S3150C0005006BCA5F6B002F0B01004600500500010003
S3150C00051003002001002F0501002F0301002F02010B
S3150C000520002F0101002F000110B54FF00053044CB1
S3150C0005300FCB84E80F00FFF7BFFEFFF729FF10BDB6
S3150C000540C4FF032008B502F0D3FE08BD2DE9F04127
S3150C00055084B04FF480330293002404AD05F80C4D9F
S3150C000560DFF8D880404609212A4600F0ABF98DF811
S3150C0005700440304E304604212A4600F0A3F98DF88B
S3150C0005800440304602212A4600F09CF98DF80440BE
S3150C000590304603212A4600F095F98DF80C40882741
S3150C0005A08DF80470304605212A4600F08BF98DF83B
S3150C0005B00C408DF80470304608212A4600F082F96A
S3150C0005C08DF80C408DF80470304609212A4600F04F
S3150C0005D079F98DF80440404608212A4600F072F954
S3150C0005E08DF80C408DF80470304607212A4600F031
S3150C0005F069F98DF80440304621462A4600F062F926
S3150C00060030462146012200F089FD4FF0806364F3E9
S3150C000610010364F38303022262F3092362F38B233F
S3150C00062064F38F33012262F39753034A136004B0C9
S3150C000630BDE8F0810082024840400050008F02481D
S3150C00064010B5244C204600F043FC2268136823F4B2
S3150C0006508013136002F04CFE00F59C54083405E040
S3150C00066002F046FEA04207D203F028F819480021F2
S3150C00067000F02AFD0028F3D0164C20460021164A1D
S3150C00068000F0F6FC2268136843F490431360236869
S3150C00069041F21802995841F400519950196841F0E9
S3150C0006A0080119602368995841F0020199501A689B
S3150C0006B042F004021A60094B08221A7000225A7082
S3150C0006C027229A706922DA705B221A7145225A71B6
S3150C0006D010BD00BF4088FE1F744000088488FE1FB2
S3150C0006E00823037000234370272383706923C37088
S3150C0006F05B23037145234371704700BF10B509484E
S3150C00070000F07EFB0446421E40F2F3539A4205D893
S3150C00071004480549224600F041FB00E0002420462F
S3150C00072010BD00BF4088FE1F1093FE1F284B1B8870
S3150C000730013B9BB240F2F352934248D8254B5A697F
S3150C00074093F826305B01D118D358002B0ADA214BCB
S3150C0007501B68022141F214029950002141F2040255
S3150C000760995070478968002303E01B4AD25CCA542F
S3150C0007700133174A12889A42F7D8164B596993F8DF
S3150C000780260001EB40114A6093F8262083F82820B6
S3150C00079058695201815841F00041815093F8262046
S3150C0007A00132D2B283F8262093F825309A4203D12F
S3150C0007B00022084B83F82620064B00221A621B687F
S3150C0007C0022041F21401585041F204015A5070476C
S3150C0007D07C92FE1F4088FE1F1093FE1F5022014B79
S3150C0007E01A6070475455000C024B1860043319609C
S3150C0007F0704700BFF055000C10B4064AAA231360CC
S3150C000800552405490C60A021116003605DF8044B6A
S3150C000810704700BF5455000CA8AA000C30B4074B07
S3150C000820AA241C60064A5521116080251D601C6097
S3150C00083011603023036030BC704700BF5455000C68
S3150C000840A8AA000CF522014B1A6070475455000CEF
S3150C00085041F21003014AD058704700BF00100058EF
S3150C00086070B506460D46FFF7EDFFFFF7B7FF002400
S3150C00087007E0631C55F8240055F82310FFF7B4FF66
S3150C00088002343F2CF5D93046FFF7B6FF41F2100380
S3150C000890024AD35813F0010FF8D170BD001000585E
S3150C0008A010B50446FFF7CEFF2046FFF7B7FF41F21F
S3150C0008B01003034AD35813F0010FF8D110BD00BF33
S3150C0008C000100058F0B48B081F1D50F8276001F07B
S3150C0008D00305ED00F824AC4026EA040440F8274052
S3150C0008E0466F4F000324BC4026EA04044467184CA8
S3150C0008F0A04203D004F58074A04207D1046E0126F1
S3150C00090006FA01F124EA0101016617E054688C40ED
S3150C0009104460CC08103450F8247001F007018900AB
S3150C00092007268E4027EA060640F8246050F8247005
S3150C000930167A06FA01F1394340F82410043350F8BC
S3150C00094023101278AA400A4340F82320F0BC7047C3
S3150C000950008E0248030F20F0704003EB43039B000C
S3150C000960014A9850704700BF14440050034B186856
S3150C000970034B5B6903F00103D8407047C0FF0320AB
S3150C00098000460050014B5860704700BF00460050AF
S3150C000990030F20F0704003EB43039B00014A985071
S3150C0009A0704700BF484600502DE9F04142F2107ED8
S3150C0009B00027BC46012638E00B6803EB83035B007B
S3150C0009C0B3FBF6F34D68B3FBF5F4374AA2FB04828E
S3150C0009D0D20802EB82025200A21A052A05D9324A23
S3150C0009E0A2FB0442D208013203E02F4AA2FB0442C6
S3150C0009F0D2082AB102EB82046400B3FBF4F304E0E0
S3150C000A00294AA2FB0323DB080122AB4201D35B1B61
S3150C000A1000E0EB1A142A07D89E4505D9B3F57A7F60
S3150C000A2006D39E461746B4460136402EC4D901E07D
S3150C000A301746B44642F2107E0126402212E042F2DC
S3150C000A40107302FB0333B3FBF7F30C899C4201D8FA
S3150C000A501D1B00E0E51AAE4501D9AE461646A3426B
S3150C000A6002D3013A022AEAD8BB1B026842F04002C2
S3150C000A700260023B1B0303F4E0434A89013A9201EC
S3150C000A80D2B21343721E120202F4706213430CF1BB
S3150C000A90FF3C0CF03F0C43EA0C030361036823F0A4
S3150C000AA040030360BDE8F081CDCCCCCCD0F8C4318A
S3150C000AB013F4407FFAD10131120442F0020242EAE9
S3150C000AC00161C0F8C411704738B50446074D284675
S3150C000AD0FFF75EFF2846FFF73DFF236823F001036F
S3150C000AE02360236813F0020FFBD138BD10000010F1
S3150C000AF0D0F8C83123F00F031943C0F8C81170475A
S3150C000B00D0F8C80100F00F00704700BF08B5FFF71A
S3150C000B10F7FF012802D0022803D005E0FFF726FFD5
S3150C000B2008BDFFF7EBFB08BD002008BDF8B5044671
S3150C000B300E461546FFF7C8FF20463146FFF7D8FF8D
S3150C000B402046FFF7E3FFB0FBF5F2C2F58062002A00
S3150C000B5038BF002240F2FF37BA4228BF3A46C2F5E8
S3150C000B608061B0FBF1F1AE098009B602B6FBF0F379
S3150C000B70BB4228BF3B4603FB00F0800A691AA5EB73
S3150C000B80801081428CBF0020012000B1134608B1B1
S3150C000B90012100E00221E26822F4434222F0FF0226
S3150C000BA0E260E26843EA81331343E360F8BD00BFB9
S3150C000BB0037E012B17D103682022DA6101680B68CA
S3150C000BC023F07062037B1B0603F0706313430B6008
S3150C000BD0036802691A61036842695A610368034A29
S3150C000BE0DA61002070470320704700BF40002800E0
S3150C000BF0026802F13843A3F5A833990AC3F34413E8
S3150C000C001B0243EA4133916821F47F4191600268EB
S3150C000C1091680B439360037E012B2FD810B50368A4
S3150C000C202022DA61C37913F0200F0ED1426802F04C
S3150C000C30604343EA824302689361826802F0604330
S3150C000C4043EA82430268D36005E0036842689A610E
S3150C000C5003688268DA600446037E012B06D1FFF72F
S3150C000C60A7FF23684FF00062DA6103E003684FF4D4
S3150C000C700062DA612368024ADA6110BD704700BF70
S3150C000C804000A0060268D169D369C3F3002311F0B2
S3150C000C90200F05D033B94FF0E063D36100207047C5
S3150C000CA004207047022070470368D969DA69C2F3D9
S3150C000CB0800211F4006F0FD182B91A6902615A6968
S3150C000CC04261D969DA69C2F3C00211F0040F07D088
S3150C000CD0002AF2D10020704703207047022070478B
S3150C000CE00020704730B400221EE0016953014FF01A
S3150C000CF00044CC500169194444F2F4544C60016927
S3150C000D001944856940F2F45404FB02548C60013298
S3150C000D1090F82410914201D0144600E00024016999
S3150C000D200B4401EB4411D96090F824309342DCD883
S3150C000D300268016941F20C03D150002380F8273078
S3150C000D4030BC704730B4002318E041695A01124C8C
S3150C000D508C5041691144C56940F2F45404FB0354A8
S3150C000D608C60013390F82510994201D01C4600E0A6
S3150C000D70002441690A4401EB4411D16090F8252006
S3150C000D809A42E2D80268416941F21003D15000231D
S3150C000D9080F8263030BC70470000103038B5044659
S3150C000DA01546036990F8270003EB4013084699682B
S3150C000DB003F04CF9226994F827305B014FF000419F
S3150C000DC0D15094F827300133DBB284F8273094F8ED
S3150C000DD02420934202D1002384F82730236841F261
S3150C000DE014029A5812F0800F08D0802141F2140296
S3150C000DF099502268002141F20803D150284638BD8B
S3150C000E00026990F827305B01D058002808DB00F403
S3150C000E100343B3F5407F05D1C0F30D40043870474A
S3150C000E20002070474FF0FF30704700BF194B1B680E
S3150C000E30194A126902F0010293405B080168174ACD
S3150C000E40934203D808230B6100207047144A93423F
S3150C000E5003D80C230B6100207047124A934202D828
S3150C000E60002008617047104A934203D804230B6193
S3150C000E70002070470D4A934203D810230B610020C3
S3150C000E8070470B4A934203D814230B61002070471A
S3150C000E9002207047C0FF032000460050C00E160209
S3150C000EA00087930300E1F50580D1F00800C2EB0B37
S3150C000EB080B2E60E10B50420FFF764FD034C204605
S3150C000EC0FFF766FD2046FFF745FD10BD0400002028
S3150C000ED038B50446FFF7EEFF236803F580531A680E
S3150C000EE042F001021A60236803F580531B6813F065
S3150C000EF0010FF8D12046FFF799FF0546A268E16875
S3150C000F002368196423685A6423684FF480621A6054
S3150C000F10236880229A612268144941F21803D15041
S3150C000F20236803F58053124A1A602046FFF7DAFE4F
S3150C000F302046FFF707FF22684FF0FF3141F21403FA
S3150C000F40D15022686FF07C43C2F810312268C2F887
S3150C000F500C3123686FF0C022C3F8002223684FF4CB
S3150C000F600272DA6300232362284638BD040020028D
S3150C000F708020010230B405682C6904F03C0444EA74
S3150C000F80C12141EA821242F001022A610022016863
S3150C000F900C6914F0010F03D14A691A80002005E090
S3150C000FA001324FF6FE718A42F1D9022030BC7047ED
S3150C000FB010B4046863610468236903F03C0343EAD4
S3150C000FC0C12141EA821242F0030323610023026825
S3150C000FD0126912F0010F06D001334FF6FE729342DE
S3150C000FE0F5D9022000E000205DF8044B704700BFE5
S3150C000FF030B583B005460C4602220DF10603FFF709
S3150C001000B9FFA0B928462146032201ABFFF7B2FF70
S3150C00101078B9BDF80630222B0DD1BDF8043023F07B
S3150C0010200F039BB2B3F5AB5F07D0032006E0042099
S3150C00103004E0042002E0032000E0002003B030BDF1
S3150C00104030B583B005460C4600224FF40043FFF73B
S3150C001050AFFF034653B92846214600220DF106037D
S3150C001060FFF788FFBDF90630002BF4DB03B030BD6B
S3150C00107070B506460D461446FFF7BAFF034608BB85
S3150C00108030462946FFF7DCFF0346D8B96388B3F52B
S3150C001090804F01D0002301E04FF40053A288B2F533
S3150C0010A0006F01D143F48073A2790AB143F48053E3
S3150C0010B0E2790AB143F48043304629460022FFF711
S3150C0010C077FF0346184670BD00B583B001220DF1BB
S3150C0010D00603FFF74FFFBDF8063003F004039BB27F
S3150C0010E00BB1012000E0002003B05DF804FB00BF4B
S3150C0010F030B48B08043350F8235001F00301C900B7
S3150C001100F8248C4025EA040440F8234050F8234088
S3150C0011108A40224340F8232030BC704710B4436FFA
S3150C001120490003248C4023EA04034367436F8A4037
S3150C0011301A4342675DF8044B704700BF70B505460D
S3150C0011400E4600F0F5F8F47904B9102428463168F7
S3150C001150224600F047F8B379013B640801342402B7
S3150C00116044EA430343F4403343F00103EB6333791E
S3150C001170013B1B0643F481736B6373792BB16A6B6A
S3150C001180013B42EA03436B6305E06A6B3379013B2F
S3150C00119042EA03436B634FF4A063AB634FF0FF3338
S3150C0011A0EB6433892B6470BDD0F8083113F0E06F13
S3150C0011B009D1836B13F0800FFBD14FF40053C3643A
S3150C0011C0C0F880107047C0F880117047D0F80C3109
S3150C0011D013F0E06F02D1406D80B27047D0F81C015D
S3150C0011E080B2704763293BD9002A3BD02DE9F041E8
S3150C0011F015460C460646FFF7B9FB1B49A1FB003703
S3150C0012007F09A1FB0431480940F2FF3E4FF0010C67
S3150C001210E046714611E001FB07F305FB00F2B3FB58
S3150C001220F2F39C0AC3F30903B4F5806F04D2734539
S3150C00123002D29E46A446884601390029EBD148F4D1
S3150C001240004333617269094B1340013D43EA852320
S3150C0012500CF1FF3C43EA0C4373610020BDE8F081BE
S3150C00126001207047012070471F85EB51EF8000FC71
S3150C00127030B4D0F8084124F0E064C0F80841D0F846
S3150C0012800851064C2C4041EA032343EA026244EA25
S3150C0012900203C0F8083130BC704700BFC0C0FFF86D
S3150C0012A030B4D0F80C4124F0E064C0F80C41D0F80E
S3150C0012B00C51074C2C4041EA032343EA026244EAF0
S3150C0012C0020343F08053C0F80C3130BC704700BFAA
S3150C0012D0C0C0FFEF10B5114B984208D14FF4006017
S3150C0012E0FFF756FB4FF40060FFF734FB10BD0C4BB9
S3150C0012F0984207D10B4C2046FFF74AFB2046FFF7D6
S3150C00130029FB10BD084B984206D1084C2046FFF726
S3150C0013103FFB2046FFF71EFB10BD00BF0800034035
S3150C0013200800024880000010084002480001001026
S3150C00133010B50446154B984203D003F5007398423A
S3150C00134003D11348FFF7C6FF14E0124B984203D0A3
S3150C00135003F50073984203D10F48FFF7BBFF09E072
S3150C0013600E4B984203D003F50073984202D10C48F9
S3150C001370FFF7B0FF0323E360E36813F0010FFBD024
S3150C001380236C23F00F03236410BD00BF0000034041
S3150C00139008000340000002480800024800400248CA
S3150C0013A008400248704700BF10B4013A0A440BE0EB
S3150C0013B00C784B7803EB04239BB2184480B298420A
S3150C0013C001D2013080B202319142F1D307D10B78B0
S3150C0013D01B02184480B2984201D2013080B25DF8EB
S3150C0013E0044B704770B4C5780D44EDB2134CE570E0
S3150C0013F083780E0A3344DBB2A370427862700078AD
S3150C00140020709CB2A64206D90132D2B20B4C627045
S3150C0014100AB901302070C9B28D420CDA0133DBB245
S3150C001420064A93703BB953780133DBB2537013B948
S3150C00143013780133137070BC704700BF8492FE1F83
S3150C00144010B50146074C20680830FFF7CBFF236820
S3150C001450054A117819725178597291789972D27825
S3150C001460DA7210BD9492FE1F8492FE1F00221A4B54
S3150C0014701A7006E00021194A22F813100133164A95
S3150C0014801370154B1B78002BF4D00022124B1A70DC
S3150C00149008E06822124902FB03120021517601333F
S3150C0014A00D4A13700C4B1B78002BF2D04FF4806254
S3150C0014B00C4B1A800022084B1A7007E00A4A02EB02
S3150C0014C08312002191800133034A1370024B1B785F
S3150C0014D0002BF3D0704700BF8C88FE1F0093FE1FB5
S3150C0014E09892FE1F8088FE1F5499FE1F00220A4BFD
S3150C0014F01A700BE01946094A32F813201AB9074B31
S3150C00150023F8110070470133034A1370024B1B7802
S3150C001510002BEFD0704700BF8C88FE1F0093FE1F78
S3150C001520030A43EA002080B2704700BF08B50020CA
S3150C00153005491422FFF738FF10B1FFF7F1FF08BD7C
S3150C0015404FF6FF7008BD00BF1E93FE1F38B50D4D3C
S3150C0015502C7C6B7C03EB0424143CA4B2204480B298
S3150C00156005F11A010822FFF71FFF05F12201224699
S3150C001570FFF71AFF10B1FFF7D3FF38BD4FF6FF7018
S3150C00158038BD00BF1093FE1F08B50620FFF7DEFF1F
S3150C00159008BD00BF70B5A54B1C68042800F071810E
S3150C0015A0A34BA44A1360A44A1360032810D1637E8C
S3150C0015B003F00F03032B40F0DA85238A002B40F04F
S3150C0015C0D68508229D4B1A7002F090F900F094BC57
S3150C0015D002287BD19A4AD3780133DBB2D37063B934
S3150C0015E093780133DBB293703BB953780133DBB29A
S3150C0015F0537013B91378013313700023914A138077
S3150C001600914A1380637E072B01D0052B0AD1A37E4A
S3150C0016100133DBB2A376782B40F0A98500236376E1
S3150C00162000F0A5BD002B00F0A285228A002A41D02D
S3150C001630A27E511EA176002A40F09985E27E082AE8
S3150C00164005D0591EC9B201290ED8052A0CD1002382
S3150C00165063768022794B1A7002F048F914227B4B80
S3150C00166083F82F2000F014BD042A03D803219140DF
S3150C001670C9B200E03021A1760132E27603F00F0305
S3150C001680013B072B00F27385DFE813F078020800A4
S3150C0016900D00F2037105F2037105F20300226B4B88
S3150C0016A083F82F206EE20422644B1A7002F01EF9A6
S3150C0016B000F057BC03F00F03032B40F058850822AB
S3150C0016C05E4B1A7002F012F900F016BC052817D101
S3150C0016D05F4B1B689B88002B00F049850023534AFF
S3150C0016E013605C4A53490A6053490A60564A138090
S3150C0016F0544A13800822514B1A7001F04DFAC0E07F
S3150C001700524B9B7B452B40F03285504A157C537CC3
S3150C00171003EB05214B4A1288914200F328858DB2C2
S3150C001720484B1D80494B1B7D13F03F0F40F01F8526
S3150C001730464B5B7D002B40F01A85474B1C880CB939
S3150C0017405B885BB1414BDB8B9C4240F010853F4B79
S3150C0017501A8C414B5B889A4240F00985FFF7E6FEEE
S3150C0017604FF6FF73984240F00285384BDB7D062B13
S3150C00177000F0B880112B23D0012B40F0F884334BAA
S3150C00178093F82230082B40F0F284304B002283F879
S3150C00179022209B8C4FF6F672934203D909332B4ABF
S3150C0017A0938402E00833294A9384284B5A8BDA83B4
S3150C0017B09A8B1A845C83284A52889A8300F0D3BC8D
S3150C0017C01C3D204B1D80254A214B1A6026E09A8829
S3150C0017D00AB31E49898C8A421DD1DA8832B11B495B
S3150C0017E0498C8A4202D0B2F58A4F14D11A8812B9A2
S3150C0017F05988002936D04FF6FF718A4202D1588893
S3150C00180088422FD01149498B8A4204D10F4A918BB9
S3150C0018105A88914226D040330D4A13600C4B1B68F4
S3150C0018200F4A9342D3D300F0A2BC00BF9492FE1F82
S3150C0018304693FE1F9092FE1F8092FE1F8892FE1FFB
S3150C0018407C88FE1F7C92FE1F5299FE1F1093FE1F72
S3150C0018508C92FE1F3A93FE1F0C93FE1F5499FE1F8B
S3150C0018609499FE1F0023AD4A13600221AC4A1170F5
S3150C001870AC4AAD490A60AD490A60AD4A138001F025
S3150C0018808BF9AB4B1A88002A00F0718402F11C010B
S3150C00189089B2A84B1980A84B080A18745974A74921
S3150C0018A00968087A98751120D875083292B2100A10
S3150C0018B040EA0222DA84002283F8282083F82920C1
S3150C0018C08A885A84CA889A849D4A10885883528872
S3150C0018D09A830A88DA834A881A843633924A1360C2
S3150C0018E000F02CBCFFF750FE4FF6FF73984240F009
S3150C0018F03E84944C17E0617EA1B18F4B9A8CA388E1
S3150C0019009A420FD18C4B5A8CE3889A420AD18A4B55
S3150C0019105A8B23889A4205D1874B9A8B63889A42B5
S3150C00192000F04A816834874B9C42E4D9824B93F889
S3150C0019302F3003F03F03022B14D17F4B9B8C99B2B3
S3150C001940814A13800022814B1A7007E0804A32F8D4
S3150C001950132091425BD001337C4A13707B4B1B786E
S3150C001960002BF3D0744B93F82F3013F0040F40F088
S3150C001970FE83714B142283F82F2028216D4A118087
S3150C001980502283F82E2093F8290093F82D2083F803
S3150C001990292093F8281093F82C2083F8282083F814
S3150C0019A02C1093F8272093F82B4083F8274083F8C4
S3150C0019B02B2093F82640654D2C7093F82A5083F80B
S3150C0019C0265083F82A400130C0B283F82D0068B93E
S3150C0019D04B1CDBB2584981F82C303BB9531CDBB29B
S3150C0019E081F82B3013B9013481F82A40524B5A8CAA
S3150C0019F055490A80998C59849A845A8BDA839A8B26
S3150C001A001A844F4A1188598352889A8381E3002499
S3150C001A104E4B1C701CE0194668224A4802FB030216
S3150C001A20527E1AB9682404FB010415E0072A0CD16E
S3150C001A303CB16822434902FB0312917EA27E91427D
S3150C001A4003D9404A682404FB032401333F4A13702C
S3150C001A503E4B1B78002BDED0002C00F088832F4BDE
S3150C001A601C600323A37623760023A3750422E27558
S3150C001A70E376314DAB8CA3806B8CE3806B8B238030
S3150C001A80AB8B638001206076324B1A7822735A78BE
S3150C001A9062739A78A273DB78E373208295F8293007
S3150C001AA0E37295F82830A37295F82730637295F88F
S3150C001AB026302372FFF7C4FC95F82E0000F0F003D5
S3150C001AC0502B5BDD0022214B1A704FE003F13602DE
S3150C001AD0194DAA5C204D2A70002A4FD0012A03D139
S3150C001AE001331A4A137041E0022A37D103F1370247
S3150C001AF0114DAA5C042A31D101F13803EA5C393163
S3150C001B006B5C43EA0222104B1A8040F20A63934242
S3150C001B1028BF13466382A38230E000BF9492FE1F57
S3150C001B208892FE1F3A93FE1F9092FE1F8092FE1F14
S3150C001B305299FE1F7C92FE1F1093FE1F8C92FE1F65
S3150C001B400C93FE1F9892FE1F7888FE1F8C88FE1F32
S3150C001B500093FE1F7C88FE1F8D88FE1F03F1370243
S3150C001B60A7498A5C52B11344A64A1370A54B1B783D
S3150C001B7019460209053AB3EB820FA7DB1022A04BDC
S3150C001B8083F82F209E4B93F82F2042F0020283F805
S3150C001B902F20022283F83620042283F837200622CF
S3150C001BA083F838200A2283F839202C21964A118092
S3150C001BB0602283F82E2072E2944B1C600022944B18
S3150C001BC01A708F4B93F82F2012F0040F07D00023B6
S3150C001BD0637620228E4B1A7001F088FEC7E2884B82
S3150C001BE093F82E301B099B0086480370EB1A143BA6
S3150C001BF09BB28548038001F00F01022903D102F044
S3150C001C003F0112290FD013B912F0030F0BD07C4BE6
S3150C001C10D98C2389994240F03782794B198D638987
S3150C001C20994240F0318212F0100F48D0218A0029D7
S3150C001C3045D004F10C00FFF7D5FB714B93F82A3015
S3150C001C40744A107883423AD16D4B93F82B30517805
S3150C001C508B4234D16A4B93F82C30927893422ED126
S3150C001C60674B93F82D506B4BDB789D4227D1207335
S3150C001C706173A273E373E37ED3B9237EA27E9A1AB1
S3150C001C80A17DA2EBD10202F0FF02D3B21144C9B27C
S3150C001C90A17513F0800F01D05242D3B2E07DA3EBB5
S3150C001CA0900250FA82F2D3B2E37503EBD10323769A
S3150C001CB00122574B1A70237EA37600232382617E62
S3150C001CC001F00F03013B072B00F25182DFE813F002
S3150C001CD008002300AA007601A601C201DC016801F6
S3150C001CE04B4B1B7813F0010F00F0418203236376F4
S3150C001CF04022474B1A7000232382434B188820B18D
S3150C001D004222434B1A70FFF79BFB0022424B1A8070
S3150C001D1001F0ECFDF0E03E4B1B7813F0010F65D0A3
S3150C001D20374B93F82F3003F03F03122B5ED1344B15
S3150C001D3093F82E0000F0F003502B39DD0022314BC6
S3150C001D401A702DE003F136022D4DAA5C334D2A7024
S3150C001D5072B3012A03D101332A4A137020E0022AF6
S3150C001D6016D103F13702264DAA5C042A10D101F1D3
S3150C001D703803EA5C39316B5C43EA0222284B1A8041
S3150C001D8040F20A63934228BF13466382A3820FE094
S3150C001D9003F137021A498A5C52B11344194A13707B
S3150C001DA0184B1B7819460209053AB3EB820FC9DBAF
S3150C001DB003236376124B93F82620227293F827207E
S3150C001DC0627293F82820A27293F82930E3720120EC
S3150C001DD0FFF736FB42220E4B1A70002323820A4A67
S3150C001DE013800D4A138001F081FD85E02022084BFB
S3150C001DF01A7001F07BFD054B1B6800225A76B1E583
S3150C001E001093FE1F8C88FE1F7C92FE1F9492FE1F61
S3150C001E108892FE1F8492FE1F5299FE1F8D88FE1F0C
S3150C001E207888FE1F914B93F82F3013F0010F24D0B6
S3150C001E3011F0100F21D1238A002B40F098818C4D84
S3150C001E402888013080B2FFF7FBFA8A4A137843F0F0
S3150C001E50100313702A881AB143F00203854A1370D3
S3150C001E6001F044FD01232382082363760023E376E5
S3150C001E7011227E4B83F82F200AE113F0200F10D08D
S3150C001E807A4890F834301A0290F8353042EA03005A
S3150C001E90794D2E6830442860754813430288D31A4E
S3150C001EA00380734B188848B111F0100F06D1714A94
S3150C001EB0137843F002031370FFF7C2FA6B4A92F8D9
S3150C001EC0301092F8313003EB01239BB26B4A13802E
S3150C001ED0A28A934200D80BB9684B1A80674B1B88B1
S3150C001EE06382644B1B7813F0030F00F040810022D1
S3150C001EF0634B1A8001F0FAFC5E4B1B7813F0200F33
S3150C001F0008D000235E4A138063761422574B83F85D
S3150C001F102F20BDE013F0100F0CD00023584A13806D
S3150C001F200122228204226276E37611224F4B83F839
S3150C001F302F20ADE0524A12888AB113F0010F01D05E
S3150C001F4000232382238A43B9638A9A4201D94C4AD5
S3150C001F5013804B4B1B88238201E0494A13800023D4
S3150C001F60E376484B1A68444B1A60454B1B884BB1B9
S3150C001F70238A3BB128333E4A138018223B4B83F805
S3150C001F802F2088E03B4B1B7813F0020F00F0EF80FC
S3150C001F902822374B1A801022344B83F82F207AE0F4
S3150C001FA0344B1B7813F0010F00F0E18000236376AD
S3150C001FB01022304B1A7001F099FCD8E02C4B188883
S3150C001FC008B1FFF73DFA294B93F82F3013F0010FA8
S3150C001FD015D0284B1B7813F0010F05D00723637619
S3150C001FE00023A376238201E0062363760120FFF704
S3150C001FF027FA10221F4B1A7001F078FC44E01D4B97
S3150C0020001B7813F0010F04D005236376002323827B
S3150C002010ADE0174B1B88002B36D1A8E0144B188863
S3150C00202008B1FFF70DFA114B93F82F3013F0010F8F
S3150C0020300CD0072363760023A3760120FFF700FA62
S3150C00204010220C4B1A7001F051FC1DE0084B1B883A
S3150C002050D3B98CE0074B1B7813F0010F00F0878087
S3150C002060072363760023A37681E000BF1093FE1F3F
S3150C0020707C92FE1F8892FE1F9092FE1F7888FE1F90
S3150C0020805299FE1F8092FE1F10223C4B83F82F2084
S3150C00209028223B4B1A805022384B83F82E20227A6A
S3150C0020A0364B83F82A20627A83F82B20A27A83F89F
S3150C0020B02C20E27A83F82D20227B83F82620627B63
S3150C0020C083F82720A27B83F82820E27B83F829203B
S3150C0020D00622DA75A2885A84E2889A84294A1188DB
S3150C0020E0598352889A832288DA8362881A84637E9B
S3150C0020F013F0100F06D0214B002283F8312083F801
S3150C002100302006E01D4B062283F830200A2283F885
S3150C00211031201A4C4023A375194B1B881A0A2274BA
S3150C0021206374002384F8353084F8343084F8323004
S3150C00213084F83330FFF728FAC04360860F4C4523EA
S3150C002140A3730022E273627522750F490B88013363
S3150C0021509BB20B80190AA174E37422766276FFF7A0
S3150C002160E5F9C04320830022084B1A7070BD00238A
S3150C002170034A1380054A137070BD00BF1093FE1FEF
S3150C0021807C92FE1F0C93FE1F7A88FE1F8892FE1F00
S3150C002190F8B505460E46284A138801339BB21380C0
S3150C0021A0B3F5FA4F03D34FF48052234B1A80002217
S3150C0021B0224B1A700CE0224B03EB84139F881E4BA8
S3150C0021C01888FFF7ADF98742E5D001341B4B1C701C
S3150C0021D01A4B1C78002CEED000221A700BE0184A11
S3150C0021E002EB831292881AB9154800EB831007E0AC
S3150C0021F00133124A1370114B1B78002BEFD00020C1
S3150C002200C0B10D4B1A88130A43EA02238380C68099
S3150C0022104DB90346002203F8012B4270013303F833
S3150C002220012B1A7003E02B8803806B8843804023B4
S3150C0022300372F8BD0020F8BD8088FE1F8C88FE1F37
S3150C0022405499FE1F00290CDD08B503468AB20549D0
S3150C0022500A8005490868834202D0194601F0F6FE49
S3150C00226008BD70475299FE1F8092FE1FF0B40022E3
S3150C0022703B4B1A703B4D1EE03A4C5A001A449200E6
S3150C002280A518A45AA4B103EB43029200354F3A4465
S3150C00229052886AB10788BC420AD14488A24207D147
S3150C0022A00C686C60898829812F4B1B78AB7254E0C3
S3150C0022B001332B4A13702A4B1B78072BDCD90022CF
S3150C0022C0274B1A700FE0274C5A001A449200A51897
S3150C0022D0A25A2AB903EB430292002244528832B125
S3150C0022E001331F4A13701E4B1B78072BEBD9082B97
S3150C0022F028D100231D4A13701D4A1370184A1370F7
S3150C00230013E0194A157803EB4304A400194A224436
S3150C0023109278AE1A154C2478A64203DD134A167031
S3150C002320134A137001330E4A13700D4B1B78072B8F
S3150C002330E7D90F4B1D780A4B1D7005EB45039B0027
S3150C002340084D1D4402682B4643F8042B0A686A6044
S3150C0023508A889A80044B1B78AB72F0BC704700BF1E
S3150C0023608E88FE1F9088FE1FF188FE1F8F88FE1F29
S3150C002370F088FE1F9888FE1F70B4174B1878013032
S3150C002380C0B218700022154B1A701EE014495A0080
S3150C0023901A4492008C18895A62880A4312D003EBAD
S3150C0023A0430189000F4A0A449278821A772A09DD7A
S3150C0023B00B4E0C467518002131556970AA1C02F893
S3150C0023C0011B11700133054A1370044B1B78072B44
S3150C0023D0DCD970BC704700BFF188FE1F8E88FE1FCB
S3150C0023E09088FE1F9888FE1F38B5354B1B88292B05
S3150C0023F003D80022324B1A8038BD0022304B1A808B
S3150C002400304B9B8AB3F5807F03D0B3F5007F44D065
S3150C00241038BD2C4BDA8C2C4B1B889A424ED1294B4F
S3150C0024201A8D294B5B889A4248D1284CA51F204609
S3150C0024302946FFF71BFFA4F11C03002204F8082C05
S3150C002440022204F8072C54F8061C616034F8021CAE
S3150C00245021811F49086844F8060C898824F8021C57
S3150C00246044F8160C24F8121C616844F81C1C2289CA
S3150C00247024F8182C9A8B62816288A281124A1188E0
S3150C002480998352886280082204F8102C062204F8DC
S3150C0024900F2C2A220A4B1A8038BD0A4BDA8C0A4BAF
S3150C0024A01B889A420AD1074B1A8D074B5B889A42B6
S3150C0024B004D1064908460639FFF7D8FE38BD00BFD9
S3150C0024C07C92FE1F1093FE1F0C93FE1F2C93FE1F77
S3150C0024D08488FE1F10B5514BD98B8AB24FF6FF7309
S3150C0024E09A420CD14D4B188C4FF6FF73984206D17D
S3150C0024F04A4B4B4A1068186092889A807EE0494B8A
S3150C0025001B88494800885340184209D1434B1A8C02
S3150C00251094B2444B5B88444840886340184206D0CA
S3150C002520424B434A1188198052885A8002E03F4B2D
S3150C00253019805A8000223F4B1A703F4C16E03E49D8
S3150C0025405A001A4492008C18384800888A5A9042CD
S3150C00255009D1364A518803EB4302920036480244AD
S3150C0025605288914206D00133324A1370314B1B7894
S3150C002570072BE4D9082B3BD1284C2046FF210622F9
S3150C00258001F06FFD002384F8203084F8213084F8A4
S3150C002590223084F8233084F8243084F82530274AF6
S3150C0025A01168C4F8061092886281C4F8161062830A
S3150C0025B01E4A1188E184528822851A4A1188A18301
S3150C0025C05288E283237501226275A373E273082293
S3150C0025D0227463740623A3740423E3742273062300
S3150C0025E063733634164B1C602A22164B1A8010BDA8
S3150C0025F00A4B54F8042F1A60A2889A80074B0F4A8C
S3150C0026001168C3F8061092885A8108221A730022A0
S3150C0026105A730C4A13880E33138010BD1093FE1F89
S3150C0026207C4000080C93FE1F0893FE1FF488FE1FC7
S3150C0026300493FE1F8E88FE1F9088FE1F8488FE1F43
S3150C0026409092FE1F7C92FE1F10B504464160FDF76A
S3150C00265079FF206010BD00BF10B50446FDF772FF70
S3150C0026602368C01A63689842B4BF0020012010BDCD
S3150C002670352303700123437081700330704700BF0C
S3150C00268003463622027004224270034A1068C3F8CD
S3150C0026900200981D704700BF1489FE1F3723037074
S3150C0026A00323437001228270C37006230371053025
S3150C0026B0704700BFFF23037001307047074B828CB5
S3150C0026C01A80C28C5A80064B028D1A80428D5A8013
S3150C0026D0044B028E1A80428E5A8070470C93FE1F52
S3150C0026E00893FE1F0493FE1F034632220270042237
S3150C0026F04270034A1068C3F80200981D704700BF69
S3150C0027001C89FE1F10B40346014400242EE01A78DF
S3150C002710332A24D006D8032A10D0062A13D0012A2D
S3150C00272021D106E0362A15D0FF2A21D0352A1AD116
S3150C0027300EE0D3F80200104A906214E0D3F80200BF
S3150C0027400D4A10630FE0D3F802000B4AD0620AE080
S3150C0027509C7808E0D3F80200074AD06103E0D3F86E
S3150C0027600200054A10625A78023213448B42CED3C9
S3150C00277020465DF8044B7047F888FE1FF8B50446F2
S3150C0027800123037043701C4B9A6982700025C57037
S3150C0027901A4A10686060258180276781184A12687A
S3150C0027A0E26025746574A574E57425756575A57563
S3150C0027B0E57525766576A576E5769E6904F11C00A9
S3150C0027C05969324601F042FCA0191C302946C6F163
S3150C0027D0100201F046FC04F12C002946402201F0BF
S3150C0027E040FC04F16C0029463A4601F03AFC054BD4
S3150C0027F01868C4F8EC00F8BDF888FE1F8440000881
S3150C0028000C93FE1F8840000838B50A4C25682846EC
S3150C002810FFF7B4FF05F1F0000121FFF729FFFFF7E1
S3150C0028203DFFFFF747FF2368C11A1846FFF70AFD5D
S3150C00283038BD00BF9092FE1F38B50B4C2568284654
S3150C002840FFF79CFF05F1F0000321FFF711FFFFF7DF
S3150C00285017FFFFF749FFFFF72DFF2368C11A18462C
S3150C002860FFF7F0FC38BD00BF9092FE1F10B5114B60
S3150C0028701C682378022B17D1201D0F49042201F066
S3150C002880D5FB98B90D4B04F11C0059699A6901F0F6
S3150C002890CDFB68B92069094B586204F1F000084B6E
S3150C0028A01988FFF72FFF10BD002010BD002010BDAA
S3150C0028B0002010BD9092FE1F84400008F888FE1F71
S3150C0028C07C92FE1F10B582B00C4C6061A161002396
S3150C0028D0A3704FF6FF73ADF80430ADF8063001A8BF
S3150C0028E04FF48641FFF754FC606010B14FF48843F7
S3150C0028F083800022014B1A8002B010BDF888FE1F9F
S3150C002900024B00221A805A80704700BF0C93FE1FA0
S3150C00291038B59E4B1B88B3F5937F7FD010D840F209
S3150C0029200F12934234D0B3F5887F01D2EBB118E184
S3150C002930B3F5887F34D040F22512934266D010E16D
S3150C002940B3F5AB7F00F0BF8005D840F25512934229
S3150C00295000F0B28005E1B3F5B57F00F0CE8040F211
S3150C0029606B12934200F0D080FBE0884B01229A70E8
S3150C0029704FF47A721A61FFF747FF844C04F1080092
S3150C0029802169FFF761FE40F20F132380002300E05C
S3150C0029900123002B00F0EA804FF488727B4B1A80DF
S3150C0029A07B4B1B7813F0020F05D17A48FFF754FEC8
S3150C0029B0002800F0DD80764B1B7813F0020F07D051
S3150C0029C0FFF754FF022803D10222704B9A700CE0D9
S3150C0029D06E4B1B694EF65F22934202DC5B006B4A20
S3150C0029E013616A4B9B78022BC5D14FF47A72674BF5
S3150C0029F01A61FFF721FF654C04F108002169FFF706
S3150C002A0023FE40F225132380002300E00123002B34
S3150C002A1000F0B0804FF493725C4B1A805C4B1B78C1
S3150C002A2013F0020F05D15B48FFF716FE002800F0E5
S3150C002A30A380574B1B7813F0020F07D0FFF716FF36
S3150C002A40052803D10322514B9A7011E04F4B1B6999
S3150C002A5042F21072934207DC4C4A03F57A73136107
S3150C002A609378032BC5D103E00020484B188038BD62
S3150C002A704648FFF723FE454D288CFEF751FD04040E
S3150C002A80688CFEF74DFD204340084FF47A7303FB28
S3150C002A9000F0002801DB286103E06FF000423B4B9D
S3150C002AA01A613A4C04F108002169FFF7CDFD40F29A
S3150C002AB055132380002300E00123002B5ED04FF436
S3150C002AC0AB72324B1A803348FFF7C6FD002857D03D
S3150C002AD02E4B02229A704FF47A721A61FFF710FF8E
S3150C002AE0FFF7AAFE294C04F108002169FFF7ACFD9B
S3150C002AF04FF4B5732380002300E00123002B41D053
S3150C002B0040F26B12214B1A80214B1B7813F0020FEB
S3150C002B1004D12048FFF7A0FD002835D01C4B1B78AC
S3150C002B2013F0020F07D0FFF7A1FE052803D10322ED
S3150C002B30164B9A7011E0154B1B6942F210729342B8
S3150C002B4007DC124A03F57A7313619378032BC7D10A
S3150C002B5003E000200D4B188038BD0C48FFF7AEFD86
S3150C002B6089E70022094B1A80022038BD032038BDA4
S3150C002B70002038BD032038BD002038BD032038BDE9
S3150C002B80002038BD032038BD002038BDF888FE1F54
S3150C002B908892FE1F0089FE1F08B5FFF7B9FE08BD17
S3150C002BA072B6704762B6704710B584B0FDF7DEFE9C
S3150C002BB0044602E0640000F081FD4C4B9C42F9D9BE
S3150C002BC002E0640800F07AFD494B9C42F9D849486A
S3150C002BD001212246FDF7AAFF0194474B02934FF4BD
S3150C002BE0FA53ADF80C300123ADF80E30434C2046A9
S3150C002BF001A9FDF7D9FE236843F04003236023683F
S3150C002C0043F0010323603E4B3E481860DA790221FB
S3150C002C1061F38712DA71596840F2E17464F31C01AE
S3150C002C2059609A6864F31C029A60090E6FF3451199
S3150C002C30D971120E42F02002DA72C26842F00052CA
S3150C002C40C26008221A73002305E02D4A1A4400219B
S3150C002C5011740133DBB2072BF7D92948012404760A
S3150C002C60FDF7C6FF234821460022FDF71FFF264B22
S3150C002C7026481860DA79022161F38712DA715968ED
S3150C002C8040F2676464F31C0159609A6864F31C0291
S3150C002C909A60090E6FF34511D971120E42F020029B
S3150C002CA0DA72C26842F00052C26008221A7300231C
S3150C002CB005E0154A1A44002111740133DBB2072BC7
S3150C002CC0F7D9114800230376FDF792FF0948012135
S3150C002CD00A46FDF7EBFE094B1A6822F040021A6011
S3150C002CE01A6822F001021A6004B010BDFF1AB70070
S3150C002CF0000E27070040014820A1070000430148A9
S3150C002D003089FE1F005001485089FE1F2050014893
S3150C002D1010B5144B1973002305E0C45C114A1A4410
S3150C002D2014740133DBB28B42F7D30E4C2046FDF7FD
S3150C002D303FFF23680222DA612046FDF7A3FF00F06D
S3150C002D40D7FA00F1320405E000F0B8FC00F0D0FA36
S3150C002D50A04205D8034B1B68DB6913F0020FF3D1B5
S3150C002D6010BD00BF3089FE1F38B5124B1B68DB69DE
S3150C002D7013F0010F1CD00D4604460E48FDF794FFC8
S3150C002D8080B90C4B1B7B2B70034606E0094A1A4490
S3150C002D90127CE2540133DBB20120064A127B9A42C2
S3150C002DA0F4D800E00020034B1B680122DA6138BD21
S3150C002DB0002038BD5089FE1F08B5FFF7F1FE08BD8F
S3150C002DC010B500F05BFA10B900F068FC10BD00F00D
S3150C002DD0C5FF10B900F062FC10BD00F01FFC00F03E
S3150C002DE05FFA00F04FFA20F0604020F07F00054BB0
S3150C002DF0186000F047FA4468FFF7D4FEA04700F0CD
S3150C002E004DFC10BD08ED00E070B508E0461C4D1CED
S3150C002E100B78037000F052FC224630462946531EAE
S3150C002E209CB2002AF2D170BD030E082B01D100F121
S3150C002E308060704738B50546002419E000F03EFC6A
S3150C002E4004EB44039B000C4AD258AA420ED804EB5E
S3150C002E5044039B00084803445B681A44AA4205D9FC
S3150C002E6004EB440189000144087A38BD0134E4B20C
S3150C002E700D2CE3D9FF2038BD8C40000838B505462B
S3150C002E80002410E000F01AFC04EB44039B00084AF3
S3150C002E9013441B7AAB4204D104EB4401890050580D
S3150C002EA038BD0134E4B20D2CECD94FF0FF3038BDEF
S3150C002EB08C40000808B5C1F3090353B903688B426B
S3150C002EC009D040F8041B4FF48062FFF79DFF0120E8
S3150C002ED008BD002008BD012008BD00BF2DE9F0414A
S3150C002EE006460068FFF7A6FFFF2833D000272CE024
S3150C002EF000F0E4FB35683C0225443444043400F00D
S3150C002F00F7F900F10D0828462146FDF7A9FC05E066
S3150C002F1000F0EEF9404520D800F0D0FBFDF798FC08
S3150C002F2000F0010010F0FF0FF2D1FDF791FC30F02C
S3150C002F30100315D1002305E0EA5CD2B2E15C8A42AB
S3150C002F4011D10133FF2BF7D90137032FD0D901202B
S3150C002F50BDE8F0810020BDE8F0810020BDE8F081DD
S3150C002F600020BDE8F0810020BDE8F08138B50446AC
S3150C002F700D460B4B984206D00A4B994205D0FFF7EB
S3150C002F80ADFF18B908E0084C00E0054C2046294670
S3150C002F90FFF790FF10B938BD002038BD204638BD6C
S3150C002FA07089FE1F0080000C748DFE1F2DE9F04108
S3150C002FB006460C4617461D4621F47F7828F0030872
S3150C002FC00368B3F1FF3F04D14146FFF773FF034695
S3150C002FD030B33368434505D030464146FFF7C6FF4C
S3150C002FE00646D0B13368E41A3444043400F066FB68
S3150C002FF0331DE31AB3F5806F07D3304608F58061AD
S3150C003000FFF7B4FF064650B1041D17F8013B04F850
S3150C003010013B013DEAD1012302E0002300E000233D
S3150C0030201846BDE8F08100BFF8B505460E46884245
S3150C0030302ED801282ED90F2926D92DE000F03EFBDB
S3150C0030402846FFF71BFF0746B0F1FF3F26D000F0DE
S3150C0030504FF900F5CE5408343846FDF721FC05E04F
S3150C00306000F046F9A0421BD800F028FBFDF7F0FB58
S3150C00307000F0010010F0FF0FF2D1FDF7E9FB30F084
S3150C00308020030FD10135EDB2B542D7D90120F8BDD9
S3150C0030900020F8BD0020F8BD0020F8BD0020F8BDCA
S3150C0030A00020F8BD0020F8BD4FF0FF33024A136034
S3150C0030B0024A1360704700BF748DFE1F7089FE1F95
S3150C0030C070B50D461646FFF7AFFE04466A1E144B46
S3150C0030D01B1A9A421ED8FFF7ADFEFF281CD06019AA
S3150C0030E00138FFF7A7FEFF2818D024F47F7323F0CE
S3150C0030F003030C4A934206D10B48214632462B4613
S3150C003100FFF754FF70BD0948214632462B46FFF7A0
S3150C0031104DFF70BD002070BD002070BD002070BD3D
S3150C003120FFFF1F0C0080000C7089FE1F748DFE1FA4
S3150C00313070B50C46FFF778FE0546621E0C4B1B1A43
S3150C0031409A420FD8FFF776FE064628190138FFF784
S3150C00315071FE0146FF2E07D0FF2807D03046FFF739
S3150C00316063FF70BD002070BD002070BD002070BDD7
S3150C003170FFFF1F0C114B1B68B3F1FF3F18D000B5B6
S3150C00318083B00E4B59689A681144DA6811441A696F
S3150C00319011445A6911449A691144DA698B18DB4354
S3150C0031A002AA42F8043D06480421FFF789FF01E014
S3150C0031B00120704703B05DF804FB00BF7089FE1F49
S3150C0031C00082000C0E4B1A6804331B6813440D4A1C
S3150C0031D0126813440C4A126813440C4A12681344BE
S3150C0031E00B4A126813440B4A12681344DB430A4A0F
S3150C0031F01268934201D1012070470020704700BF2E
S3150C0032000080000C0880000C0C80000C1080000C58
S3150C0032101480000C1880000C0082000C08B50D4BB5
S3150C0032201B68B3F1FF3F04D00A48FFF757FE03466D
S3150C00323068B1094B1B68B3F1FF3F05D00648FFF791
S3150C0032404DFE034610B902E0012300E001231846A7
S3150C00325008BD00BF7089FE1F748DFE1F00487047A5
S3150C0032600080000C08B5FFF71FFF08BD08B5FFF777
S3150C00327027FF08BD08B5FFF75BFF08BD08B5FFF7CC
S3150C003280A1FF08BD08B5FFF7E9FF08BD08B5FFF7B4
S3150C00329071FF034610B1FFF7C1FF0346184608BD80
S3150C0032A00022014B1A60704710E000E008B5FFF7EA
S3150C0032B0F7FF054B054A5A6000229A6005211960F2
S3150C0032C0034B1A6008BD00BF10E000E07F3202001D
S3150C0032D07891FE1F044B1B6813F4803F03D0034AFE
S3150C0032E0136801331360704710E000E07891FE1FFD
S3150C0032F008B5FFF7EFFF014B186808BD7891FE1F64
S3150C003300134BD3F8143113F4805F1ED110B501465C
S3150C0033100F48FDF749FFFFF7EBFF00F10A0405E044
S3150C00332000F0CCF9FFF7E4FFA04207D8084BD3F81E
S3150C003330143113F4807FF3D0012000E000204FF409
S3150C0033408072034BC3F8182110BD0020704700BFD4
S3150C00335000000340074BD3F8143113F0080F07D1C4
S3150C00336010B504460348FDF731FF2070012010BD4F
S3150C0033700020704700000340F0B585B04FF4614360
S3150C003380019308238DF808308DF8093001258DF846
S3150C0033900A5010278DF80B700026ADF80C600C4CFB
S3150C0033A0204601A9FDF7CAFE2046394604222B46C3
S3150C0033B0FDF75EFF2046314604222B46FDF770FFD3
S3150C0033C0236C23F00F0343F00203236405B0F0BD16
S3150C0033D00000034070B506460D46402903D9104837
S3150C0033E07A2100F073F82846FFF78AFF012803D0EC
S3150C0033F00B487E2100F06AF800240CE000F05EF920
S3150C003400305DFFF77DFF012803D00548872100F0CA
S3150C0034105DF80134A4B2ABB2A342EFD870BD00BFC5
S3150C0034203441000870B5244B1C78ACB92348FFF71F
S3150C00343091FF01283DD1214B1B78013BDBB23F2B81
S3150C00344037D8FFF755FF1E4B186000221D4B1A701C
S3150C0034500122194B1A702CE006460D46194B1B78A7
S3150C00346019481844FFF776FF0446012813D1154B6B
S3150C0034701A780132D2B21A70104B1B789A4215D1B7
S3150C00348030461149FFF7C0FC00220B4B1A700D4B4E
S3150C0034901B782B700DE0FFF72BFF094B1B68643371
S3150C0034A0984205D90024044B1C7002E0002400E06D
S3150C0034B00024204670BD00BFC591FE1F8091FE1FE3
S3150C0034C07C91FE1FC491FE1F8191FE1F08B500F072
S3150C0034D0F5F8FCE708B500F0DDF8012813D00A4B27
S3150C0034E01B78012B0FD1FFF703FF084B1A68084B0B
S3150C0034F01B68134403F5FA73984204D30022024B5B
S3150C0035001A70FFF75DFC08BDCC91FE1FC891FE1F1B
S3150C003510D091FE1F014B1860704700BFC891FE1F6B
S3150C003520014B1868704700BFC891FE1F08B5044BC5
S3150C0035301B78012B03D1FFF7DBFE024B186008BD8D
S3150C003540CC91FE1FD091FE1F08B50122034B1A70B9
S3150C003550FFF7ECFFFFF7BEFF08BD00BFCC91FE1FC7
S3150C00356008B5FFF729FC00F0A5F8FFF79FFEFFF75B
S3150C00357079FE00F00DF8FFF7E7FF08BD08B500F07F
S3150C0035809DF8FFF7A7FE00F013F8FFF7A3FF08BDA1
S3150C00359010B500F053FBFFF707FB044C0123237017
S3150C0035A0FFF7EAFE0023237010BD00BF7088FE1FD4
S3150C0035B000B583B017480DF10701FFF7D5FB0128BD
S3150C0035C007D10122144B1A7012489DF8071000F00F
S3150C0035D053FB10480DF10701FFF724FF012807D113
S3150C0035E000220D4B1A700B489DF8071000F044FB97
S3150C0035F008480DF1070100F06DF9012807D10322E7
S3150C003600054B1A7003489DF8071000F035FB03B004
S3150C0036105DF804FBD491FE1F7088FE1F704700BF37
S3150C00362038B505460C460C4B1B78012B02D1C9B29A
S3150C003630FFF76EFB084B1B781BB92846E1B2FFF768
S3150C003640C9FE054B1B78032B03D12846E1B200F0CB
S3150C0036501DF900F009FB38BD7088FE1F054B1B7861
S3150C003660012B05D0022B01D040207047002070475B
S3150C003670082070477088FE1F054B1B78012B05D060
S3150C003680022B01D04020704700207047082070475D
S3150C0036907088FE1F08B500F0DFFA08BD08B500F00B
S3150C0036A0E7F80322024B1A70FFF740FF08BD00BF74
S3150C0036B07088FE1F08B500F05FFB08BD08B500F06A
S3150C0036C061FB08BD10B5FDF719F848B3384A1080F0
S3150C0036D0384B9C894FF40060FDF722FF84420DD1D4
S3150C0036E00120FDF757FF324B1B88CBB1FEF7F2FEDC
S3150C0036F0FDF71CF800222E4B1A8011E02D4B9C89ED
S3150C00370040F60600FDF70CFF844209D1FEF76CFE6D
S3150C003710274B1B8823B1FDF709F80022244B1A808E
S3150C003720FFF7E6FD244B1B68984232D303F5FA7378
S3150C003730214A1360002413E0204A682303FB042368
S3150C0037401F4A13600220FDF725FF194B1B8833B166
S3150C003750FEF7C0FEFCF7EAFF0022154B1A80013477
S3150C003760002CE9D0002412E0164B03EB8413164A06
S3150C00377013600520FDF70EFF0D4B1B8833B1FEF7CA
S3150C003780A9FEFCF7D3FF0022094B1A800134002C4A
S3150C003790EAD0FFF7ADFD0D4B1B68984206D303F537
S3150C0037A01C531033094A1360FEF7E6FD10BD00BF2B
S3150C0037B07C92FE1F1093FE1F2492FE1F9892FE1FF2
S3150C0037C09492FE1F5499FE1F8C92FE1F1892FE1F98
S3150C0037D01F4B1B78002B39D110B5FCF7B7FEFFF742
S3150C0037E087FD00F5FA701B4B1860FFF781FD00F59D
S3150C0037F01C501030184B1860FDF738FE174A002382
S3150C00380013805380164A13805380164A13805380B4
S3150C0038104EF60300FDF76AFEFCF712FF124C20462B
S3150C003820FCF75EFF20460621FFF74CF8FFF768F819
S3150C003830FFF776FE42F20F73984203D842F21070ED
S3150C003840FFF768FE0122094B1A7010BD704700BFC6
S3150C0038507188FE1F2492FE1F1892FE1F0C93FE1FEA
S3150C0038600893FE1F0493FE1F1C92FE1F1492FE1F4C
S3150C00387008B50022034B1A70034B1B780BB9FFF7E4
S3150C003880A7FF08BD7188FE1F1492FE1F38B50F4B9B
S3150C0038901B78012B18D10E4B1D68EB692B6200238C
S3150C0038A005E0C45CEA1882F8244001339BB28AB264
S3150C0038B09A42F6D8111DA5F8641005F12000FEF702
S3150C0038C0C1FCEB690133EB6138BD00BF1492FE1FDE
S3150C0038D09492FE1F08B5044B1B78012B01D1FFF700
S3150C0038E0F1FE002008BD00BF1492FE1F10B5194B47
S3150C0038F01C68194B1B7813F0400F05D00123E361AC
S3150C0039000023A4F8643010BD13F0010F02D000227E
S3150C003910A4F8642013F0040F06D0B4F8641019B19F
S3150C00392004F12000FEF78EFC0B4B1B7813F0020FF4
S3150C0039300ED00A4B19880B1F402B09DC0023A4F868
S3150C0039406430074B186804390430C9B200F094F996
S3150C00395010BD00BF9492FE1F8892FE1F7C92FE1F24
S3150C0039609092FE1F0022014B5A7070472892FE1F40
S3150C003970034BFE22DA7018710222A3F8442070471A
S3150C0039802892FE1F10B5054C00232370FFF7EAFFA3
S3150C003990FF23E3700123A4F8443010BD2892FE1FC8
S3150C0039A0064BFF22DA7000221A71597859719A71F6
S3150C0039B0DA711A720622A3F8442070472892FE1F69
S3150C0039C008B50020FFF7D4FF08BD00BF084BFF2247
S3150C0039D0DA70084A9A6400221A715A719A71072190
S3150C0039E0D9711A725A729A720822A3F84420704737
S3150C0039F02892FE1F80410008044BFF22DA704268B1
S3150C003A009A640122A3F84420704700BF2892FE1F37
S3150C003A1008B53120FFF7ACFF08BD00BF38B5084C20
S3150C003A20FF23E370002525716571FFF717FEA07162
S3150C003A30E571257265720723A4F8443038BD00BFC2
S3150C003A402892FE1F38B5FFF78DFF0E4C0125257009
S3150C003A50FF23E3701023237100236371FFF7FEFD30
S3150C003A60A071FFF709FEE071FFF706FEC0F3072011
S3150C003A7020726572A5720823A4F84430FFF7F2FB96
S3150C003A8038BD00BF2892FE1F38B505464478FFF7AF
S3150C003A90E5FD0138844203DD2220FFF769FF38BDBE
S3150C003AA0084C201DA16C6A78FFF7AEF9FF23E37072
S3150C003AB06B78A26C1344A3646B780133A4F844307E
S3150C003AC038BD00BF2892FE1F38B504464578FFF76F
S3150C003AD0C5FD0138854203DD2220FFF749FF38BDBD
S3150C003AE06168084DA964281D6278FFF78DF9FF23DC
S3150C003AF0EB706378AA6C1344AB6463780133A5F856
S3150C003B00443038BD2892FE1FF8B5054617460024EA
S3150C003B1006E015F8013B1C44E4B2FFF7CFFD314635
S3150C003B204E1E0029F5D13C600120F8BD10B5084C9D
S3150C003B30FF23E3704168A06CE21DFFF7E5FF2071DF
S3150C003B4000236371A3710823A4F8443010BD00BF91
S3150C003B502892FE1F38B504460D4B9D6CFFF77EFD73
S3150C003B60411E2846621CFFF781FB18B93120FFF76E
S3150C003B70FFFE38BD064CFF23E370FFF76FFD0138DF
S3150C003B80A36C1844A0640123A4F8443038BD00BFCC
S3150C003B902892FE1F38B504464578FFF75FFD0238BC
S3150C003BA0854203DD2220FFF7E3FE38BD0F4BFF22D3
S3150C003BB0DA700122A3F84420617831B9FFF766FB6D
S3150C003BC090B93120FFF7D4FE38BD084B986CA21C77
S3150C003BD0FFF74CFB18B93120FFF7CAFE38BD6378E6
S3150C003BE0024A916C0B44936438BD00BF2892FE1FA9
S3150C003BF008B54168074B986CFFF73CFB18B93120A8
S3150C003C00FFF7B6FE08BD034BFF22DA700122A3F8BC
S3150C003C10442008BD2892FE1F08B5FFF7D1F8034BC8
S3150C003C20FF22DA700122A3F8442008BD2892FE1F59
S3150C003C3008B589B2FFF7F4FC08BD00BF054B00229E
S3150C003C401A709A6483F84320A3F844209A705A7029
S3150C003C50704700BF2892FE1F024B187800B1012056
S3150C003C60704700BF2892FE1F0022024B83F84320A8
S3150C003C70704700BF2892FE1F08B50378FF2B02D1B0
S3150C003C80FFF7E0FE50E0344A1278012A62D1C93BB4
S3150C003C90352B46D8DFE803F03345454245453F36DC
S3150C003CA03C394545454545454545454545454545C7
S3150C003CB045454545454545454545454545454545A2
S3150C003CC04545241E1B2145454527452A2D30FFF722
S3150C003CD0DBFE29E0FFF7F8FE26E0FFF78DFE23E07A
S3150C003CE0FFF724FF20E0FFF771FE1DE0FFF768FEEB
S3150C003CF01AE0FFF755FE17E0FFF744FE14E0FFF756
S3150C003D0029FF11E0FFF746FF0EE0FFF787FE0BE0F9
S3150C003D10FFF76EFF08E0FFF77FFF05E0FFF778FE81
S3150C003D2002E02020FFF724FE0B4B93F84330012BC7
S3150C003D3002D11020FFF71CFE074BB3F844100BB250
S3150C003D40002B07DD0448012380F84330033009B209
S3150C003D50FFF76EFF08BD00BF2892FE1F08B5054B86
S3150C003D605B6A13F4005F03D000F040F8012008BD35
S3150C003D70002008BD008F024808B5642000F006F844
S3150C003D8008BD00BF08B500F007F808BD014B188048
S3150C003D90704700BF7892FE1F08B5FFF7A9FA0F4BC4
S3150C003DA01B68984218D30E4B1B783BB901220C4B5F
S3150C003DB01A704FF400720B4B5A6006E00022084B47
S3150C003DC01A704FF00072074B5A60FFF791FA064BC8
S3150C003DD01B881844014B186008BD00BF7492FE1F67
S3150C003DE07A92FE1F008502487892FE1F4FF00072F1
S3150C003DF0014B5A60704700BF0085024810B5084851
S3150C003E0009218022FDF774F9064C20460D2100226B
S3150C003E10FDF76EF9236E23F40053236610BD00BF25
S3150C003E2000850248008F02482DE9F0418CB04FF016
S3150C003E3000088DF8248001260A9602258DF82C5050
S3150C003E401C4C2046042109AAFCF73CFD90278DF852
S3150C003E50187007968DF820502046052106AAFCF707
S3150C003E6031FD154AD36923F007033343D3610CAAFA
S3150C003E7002F8248D20460D21FCF724FD8DF80070E8
S3150C003E8001968DF8085020460C216A46FCF71AFD5F
S3150C003E900A4B1A6842F040021A60DA6822F00702EE
S3150C003EA02A43DA601A6822F040021A600CB0BDE8A8
S3150C003EB0F08100BF00810248000003400043014826
S3150C003EC030B583B0002502AC04F8015DFFF796FF10
S3150C003ED000F056F8FFF744FB2846214600F068F838
S3150C003EE09DF80730012B01D1FFF7D8FBFFF79CFF9C
S3150C003EF0FFF744FBFCE700BF0C4B1968C1F3072323
S3150C003F0053FA81F3C1F307421A440B0E13FA82F3E8
S3150C003F109BB2002205E005491144087903449BB283
S3150C003F200132372AF7D9584280B270470080FE1FFB
S3150C003F3008B5FFF7E1FF044B9B8F984201D0002098
S3150C003F4008BD012008BD00BF0080FE1F08B5064B4A
S3150C003F501A68064B9A4203D1FFF7EAFF10B908BD5F
S3150C003F60002008BD012008BD0080FE1FA2E742CE3E
S3150C003F7008B5FFF7C1FF014B988708BD0080FE1FEF
S3150C003F8008B5FFF7E3FF68B9074A084B1A60002328
S3150C003F9004E0064A1A44002111710133372BF8D973
S3150C003FA0FFF7E6FF08BD00BFA2E742CE0080FE1F6A
S3150C003FB038B504460D46FFF7C9FF40B1372C08D873
S3150C003FC04DB1064B1C4423792B70012038BD0020C3
S3150C003FD038BD002038BD002038BD00BF0080FE1F54
S3150C003FE070B50E4B0E4CE41AA41000251E46A542C5
S3150C003FF004D056F8253098470135F8E7FDF7D2F985
S3150C004000084C094BE41AA41000251E46A54204D000
S3150C00401056F8253098470135F8E770BD7488FE1FB1
S3150C0040207488FE1F7488FE1F7488FE1F10B50A4420
S3150C004030441E914208D014F8013F0878834201D0FF
S3150C004040181A10BD0131F4E7002010BD10B5431E3F
S3150C0040500A44914204D011F8014B03F8014FF8E7DA
S3150C00406010BD02440346934202D003F8011BFAE743
S3150C004070704700000100004000080000FFFFFFFF32
S3150C004080FFFF0000ADDE1223638253630080000C39
S3150C004090004000000200000000C0000C00400000C0
S3150C0040A0030000000000010C0040000004000000AA
S3150C0040B00040010C00400000050000000080010CCF
S3150C0040C0004000000600000000C0010C004000008B
S3150C0040D0070000000000020C0000020008000000AF
S3150C0040E00000040C00000400090000000000080C8D
S3150C0040F0000004000A00000000000C0C0000040084
S3150C0041000B0000000000100C000004000C00000066
S3150C0041100000140C000004000D0000000000180C38
S3150C004120000004000E00000000001C0C000004003F
S3150C0041300F000000433A2F576F726B2F736F667424
S3150C004140776172652F4F70656E424C545F584D43C4
S3150C004150343730305F6578747261732F54617267CF
S3150C00416065742F536F757263652F41524D434D34F1
S3150C0041705F584D43342F756172742E630000000036
S30D0C0041804F70656E424C5400B1
S3150C00418800C0005000000000080027695B450000CD
S3150C00419820300020A02F0020D0170020000000207F
S3150C0041A800000000040400000000000000000000ED
S3090C0041B804010000EC
S70508000201EF
